:02000000A62830
:0800080005288C00030E8D0099
:1000100083010B1910280D0E83008C0E0C0E0900A5
:100020007C209B1C16289B101B18632019200B1189
:100030000B289508031D2128950A12088038860090
:10004000080001301502031D2A28950A13080038FC
:100050008600080002301502031D3328950A140893
:10006000D0388600080003301502031D3C28950A8D
:100070000F0830388600080004301502031D45289B
:10008000950A100850388600080095011108C038FC
:10009000860008009601970198018E008E080319CA
:1000A000080064308E02031C5728980A51286430D7
:1000B0008E070A308E02031C5F28970A59280A30DF
:1000C0000E07960008001A084A20822016088F00A2
:1000D000170890001808910019084A201608920085
:1000E00017089300180894001B100800640064307F
:1000F0009C009C0B792808009D0B08009B143C3049
:100100009D000800960D16101B110A301602031CE4
:100110008C280A3096021B15970D17101B191714FF
:100120001B110A301702031C98280A3097021B156E
:10013000980D18101B19181408000C308400800149
:10014000840A30300402031C9F28080064009D20AC
:10015000030166008316D3308100013088008312CA
:1001600095019B01A0308B00413088003C309D0000
:10017000640088117620081564000819BC28090855
:100180009A0088157620081564000819C428090803
:0601900099001B14B828C1
:02400E00F73F7A
:00000001FF
